:020000040000FA
:0A00000000000000A3EF01F0B8D1EA
:08001800F5D19EA8FED7AD6EE4
:1000200012000B6A0A6EFF0E0A260B2200D0D8A01F
:100030001200030E096EE60E02D8F5D7096AFE0F0C
:10004000086EE86A095AD8A012000000080600D01D
:10005000F8D7800E1E1A1D50195C226E11E2226C18
:1000600019501DC019F01D6E1A501EC01AF01E6ED8
:100070001B501FC01BF01F6E1C5020C01CF0206EB8
:100080001A0E226074D01D5272E0216A1A50256E39
:100090001E18246E1A8E1E8E080E225E08E320C0E3
:1000A00021F01FC020F01EC01FF01E6AF5D72226C7
:1000B00007E0D8901E321F3220322132222EF9D78B
:1000C00024AE33D020501C5E1F501B5A1E501A5AAB
:1000D00007E2D880000E1C561B561A56800E251AB1
:1000E000216C04E01C06000E1B5A1A5A040E226EE4
:1000F0001A660DD01BC01AF01CC01BF021C01CF0EA
:10010000216A080E195E29E3222EF2D726D01ABEE4
:1001100008D0D89021361C361B361A36192EF7D740
:100120001CD021AE22D0216A0FD020501C261F5097
:100130001B221E501A2206E31A321B321C322132B5
:10014000194A0DD021AE11D01C3E0FD01B3E0DD050
:100150001A3E0BD0D8801C90EFD7196A02D02382A8
:1001600019681C6A1B6A800E1A6E25AE1A9E1C50F6
:1001700012001A50186E1E18246E1950D8A41D5063
:100180003AE019267E0E03E3195E03E336D0195ECA
:1001900031E31CC016F01BC017F0188E1E8E1C6AAF
:1001A0001B6A1A6A180E256E18321732163206E3C9
:1001B00020501C261F501B221E501A221A321B329E
:1001C0001C32252EF1D71ABE07D01C361B361A3624
:1001D000195210E01906183416E31C3E14D01B3EC9
:1001E00012D01A3E10D0D8801A321B321C32193E5F
:1001F0000AD003D02384196A02D0238219681C6AAA
:100200001B6A800E1A6E24AE1A9E1C50120019C072
:1002100025F01A501CC01AF01C6E1C3625321C32F8
:10022000236A1C36253602E32384237E06E12380DD
:10023000256A1C6A1B6A1A6A0BD0252803E0D8803D
:100240001C3206D0D8901C3202E1238201D02386D2
:1002500023B604D023A20FD023B407D07F0E1C6E88
:10026000FF0E1B6E1A6E196E23D0800E1C6E01D00D
:100270001C6A000EF6D723B0FBD7196A9F0E2560C3
:10028000EBD77E0E2564F4D79E0E255C07E0D89050
:100290001C321B321A321932252AF6D723A408D071
:1002A000D880000E19561A561B561C561CAEE0D7A5
:1002B00019501200196E000E19BEFF0E1A6E1B6E39
:1002C0001C6E06D0196E1A6A1B6A1C6A249E0AD01C
:1002D000249E1CAE07D0D880000E19561A561B5605
:1002E0001C56248E960E256E1C5209E0080E2526FB
:1002F0001AC019F01BC01AF01CC01BF011D01B5201
:100300000FE1080E255E1A5007E1080E255E195010
:1003100002E11C5010D0196A1B6E19C01AF0196A3C
:100320001BBE06D0D89019361A361B362506F8D7CC
:1003300024AE1B9E255019C01CF0196E1B501AC00C
:100340001BF01A6E1200400E236E006A4F0EAF6E45
:10035000B06A240EAC6E900EAB6E00010F0EC16E33
:10036000070EB46EC69AC00E926EE00E936EC00E6B
:10037000946E956AE80E966E5BD09EAA17D0ABA4D9
:1003800004D0AE50AE50AB881100ABA205D0AE5039
:10039000AE50AB98AB881100462A00EE49F04650AB
:1003A000E926000EEA22AECFEFFF1100F2A409D039
:1003B000F294284A292AD6CF26F0D7CF27F0817683
:1003C00011004650475C0AE0472A00EE49F04750CA
:1003D000E926000EEA22EF50456E01D04568120072
:1003E000496A466A476A9D8A9F8AF28EF28C120099
:1003F0009D9A496A466A476AAE50AE50AB98AB8840
:100400009D8A1200F29EE0CF9DF4D8CF9EF4E8CFF3
:100410009FF4F28E0001A192B36AB26AF29E9DC46B
:10042000E0FF9EC4D8FF9FC4E8FFF28E10001000CA
:1004300093968A860A0E11EC00F093968A96929013
:1004400089909292899292948994929689969298A0
:100450008998929A899A96908D9096928D92969478
:100460008D9494908B9094928B9294948B94949678
:100470008B9695908C9095928C92959E8C9E959C47
:100480008C9C959A8C9A95988C98949A8B9A94981F
:100490008B9895968C9695948C9493908A90939241
:1004A0008A9293948A94C9EC09F0346801EE49F079
:1004B000480EEE68E82EFDD7446A92DF99DFCD6AD8
:1004C000F294F28A870ED56EB16AA192A082B36AC5
:1004D000B26AD08EA292B10EB16E0101946B936B91
:1004E000926B916B3E500DEC00F0190E0DEC00F08C
:1004F000400E0DEC00F00001D6CF26F0D7CF27F04C
:1005000060DF45C02EF0B50E2E5C07E3FE0E2E5CBC
:1005100001E301D0376A17EF08F02EAE38D0376A02
:10052000840E2E5C05E12EC037F0386839682DD076
:10053000940E2E5C05E12EC037F03A683B6825D05A
:10054000A40E2E5C05E12EC037F03C683D681DD03E
:10055000B40E2E5C05E12EC037F03E683F6815D022
:10056000C40E2E5C04E12EC037F040680ED0D40ECD
:100570002E5C04E12EC037F0416807D0E40E2E5CFB
:1005800004E12EC037F04268436815EF08F0375297
:1005900004E117EF08F015EF08F0840E375CD8A4DB
:1005A000F3D0382803E12EC038F0ECD02EC039F05B
:1005B000300E385C0AE1899001014C694B694A6947
:1005C0004969919148800001DCD0310E385C0AE124
:1005D0008992010150694F694E694D699193488034
:1005E0000001CFD0320E385C0AE1899401015469D0
:1005F000536952695169919548800001C2D0330E08
:10060000385C0AE18996010158695769566955694C
:10061000919748800001B5D0340E385C0AE1899882
:1006200001015C695B695A695969919948800001C7
:10063000A8D0350E385C0AE1899A010160695F69CA
:100640005E695D69919B488000019BD0360E385CE5
:100650000AE18D9001016469636962696169919D34
:10066000488000018ED0370E385C0AE18D9201017E
:100670006869676966696569919F4880000181D0F2
:10068000380E385C0AE18D9401016C696B696A6906
:10069000696992914880000174D0390E385C0AE192
:1006A0008B90010170696F696E696D6992934880E2
:1006B000000167D03A0E385C0AE18B92010174693F
:1006C0007369726971699295488000015AD03B0E36
:1006D000385C0AE18B9401017869776976697569FC
:1006E0009297488000014DD03C0E385C0AE18B9611
:1006F00001017C697B697A69796992994880000176
:1007000040D03D0E385C0AE18C90010180697F6920
:100710007E697D69929B4880000133D03E0E385C33
:100720000AE18C9201018469836982698169929DE1
:100730004880000126D03F0E385C0AE18C9E010102
:100740008869876986698569929F4880000119D008
:10075000400E385C0AE18C9C01018C698B698A69C6
:1007600089699391488000010CD0410E385C08E102
:100770008C9A010190698F698E698D699393488085
:100780000001386815EF08F0940E375CD8A4EBEF41
:1007900007F03A2804E12EC03AF0EAEF07F02EC045
:1007A0003BF03B52D8A4EBD0300E3A5C0AE1899082
:1007B00001014C694B694A6949699191488000017E
:1007C000DCD0310E3A5C0AE18992010150694F692F
:1007D0004E694D69919348800001CFD0320E3A5C4A
:1007E0000AE18994010154695369526951699195EB
:1007F00048800001C2D0330E3A5C0AE189960101BB
:100800005869576956695569919748800001B5D074
:10081000340E3A5C0AE1899801015C695B695A69A6
:100820005969919948800001A8D0350E3A5C0AE1D7
:10083000899A010160695F695E695D69919B488081
:1008400000019BD0360E3A5C0AE18D90010164698B
:10085000636962696169919D488000018ED0370E9D
:100860003A5C0AE18D9201016869676966696569A8
:10087000919F4880000181D0380E3A5C0AE18D9446
:1008800001016C696B696A6969699291488000012C
:1008900074D0390E3A5C0AE18B90010170696F697E
:1008A0006E696D6992934880000167D03A0E3A5C98
:1008B0000AE18B9201017469736972697169929599
:1008C000488000015AD03B0E3A5C0AE18B9401014A
:1008D00078697769766975699297488000014DD08B
:1008E0003C0E3A5C0AE18B9601017C697B697A696E
:1008F000796992994880000140D03D0E3A5C0AE146
:100900008C90010180697F697E697D69929B488036
:10091000000133D03E0E3A5C0AE18C9201018469F9
:10092000836982698169929D4880000126D03F0ECB
:100930003A5C0AE18C9E010188698769866985694C
:10094000929F4880000119D0400E3A5C0AE18C9CCD
:1009500001018C698B698A698969939148800001DA
:100960000CD0410E3A5C08E18C9A010190698F69C4
:100970008E698D69939348800001EAEF07F0300E8D
:100980003A5C2AE101019131000123E2898001EE04
:1009900095F0D8903B34E926000EEA22EECF06F01F
:1009A000EFCF07F006502624026E07502720036E73
:1009B000000E2820046E000E2920056E05C04CF1A3
:1009C00004C04BF103C04AF102C049F14880010163
:1009D00091810001E9EF07F0310E3A5C2BE1010152
:1009E00091510001E8B223D0898201EE95F0D890B0
:1009F0003B34E926000EEA22EECF06F0EFCF07F0F7
:100A000006502624026E07502720036E000E282071
:100A1000046E000E2920056E05C050F104C04FF190
:100A200003C04EF102C04DF14880010191830001E5
:100A3000E9EF07F0320E3A5C2BE101019151000120
:100A4000E8B423D0898401EE95F0D8903B34E926B0
:100A5000000EEA22EECF06F0EFCF07F00650262474
:100A6000026E07502720036E000E2820046E000E31
:100A70002920056E05C054F104C053F103C052F1A2
:100A800002C051F14880010191850001E9EF07F0B2
:100A9000330E3A5C2BE1010191510001E8B623D0FD
:100AA000898601EE95F0D8903B34E926000EEA22C3
:100AB000EECF06F0EFCF07F006502624026E075067
:100AC0002720036E000E2820046E000E2920056EDC
:100AD00005C058F104C057F103C056F102C055F1EA
:100AE0004880010191870001E9EF07F0340E3A5C7C
:100AF0002BE1010191510001E8B823D0898801EE72
:100B000095F0D8903B34E926000EEA22EECF06F0AD
:100B1000EFCF07F006502624026E07502720036E01
:100B2000000E2820046E000E2920056E05C05CF121
:100B300004C05BF103C05AF102C059F148800101C1
:100B400091890001E9EF07F0350E3A5C2BE10101D4
:100B500091510001E8BA23D0898A01EE95F0D8902E
:100B60003B34E926000EEA22EECF06F0EFCF07F085
:100B700006502624026E07502720036E000E282000
:100B8000046E000E2920056E05C060F104C05FF1FF
:100B900003C05EF102C05DF148800101918B00014C
:100BA000E9EF07F0360E3A5C2AE1010191510001AC
:100BB000E8BC23D08D8002EE95F0D8903B34E92636
:100BC000000EEA22EECF06F0EFCF07F00650262403
:100BD000026E07502720036E000E2820046E000EC0
:100BE0002920056E05C064F104C063F103C062F101
:100BF00002C061F148800101918D0001EAD1370EF8
:100C00003A5C29E101019135000123E28D8202EE77
:100C100095F0D8903B34E926000EEA22EECF06F09C
:100C2000EFCF07F006502624026E07502720036EF0
:100C3000000E2820046E000E2920056E05C068F104
:100C400004C067F103C066F102C065F1488001018C
:100C5000918F0001BED1380E3A5C29E10101923139
:100C6000000123E28D8402EE95F0D8903B34E92612
:100C7000000EEA22EECF06F0EFCF07F00650262452
:100C8000026E07502720036E000E2820046E000E0F
:100C90002920056E05C06CF104C06BF103C06AF138
:100CA00002C069F1488001019281000192D1390EA0
:100CB0003A5C2AE1010192510001E8B223D08B8015
:100CC00002EE95F0D8903B34E926000EEA22EECFF2
:100CD00006F0EFCF07F006502624026E07502720BB
:100CE000036E000E2820046E000E2920056E05C03C
:100CF00070F104C06FF103C06EF102C06DF1488065
:100D000001019283000165D13A0E3A5C2AE10101AA
:100D100092510001E8B423D08B8202EE95F0D89076
:100D20003B34E926000EEA22EECF06F0EFCF07F0C3
:100D300006502624026E07502720036E000E28203E
:100D4000046E000E2920056E05C074F104C073F115
:100D500003C072F102C071F1488001019285000167
:100D600038D13B0E3A5C2AE1010192510001E8B60C
:100D700023D08B8402EE95F0D8903B34E926000E08
:100D8000EA22EECF06F0EFCF07F006502624026EDF
:100D900007502720036E000E2820046E000E292025
:100DA000056E05C078F104C077F103C076F102C08A
:100DB00075F148800101928700010BD13C0E3A5C2D
:100DC0002AE1010192510001E8B823D08B8603EE9D
:100DD00095F0D8903B34E926000EEA22EECF06F0DB
:100DE000EFCF07F006502624026E07502720036E2F
:100DF000000E2820046E000E2920056E05C07CF12F
:100E000004C07BF103C07AF102C079F1488001018E
:100E100092890001DED03D0E3A5C2AE10101925137
:100E20000001E8BA23D08C8003EE95F0D8903B34D3
:100E3000E926000EEA22EECF06F0EFCF07F00650CB
:100E40002624026E07502720036E000E2820046E11
:100E5000000E2920056E05C080F104C07FF103C09B
:100E60007EF102C07DF148800101928B0001B1D07A
:100E70003E0E3A5C2AE1010192510001E8BC23D008
:100E80008C8203EE95F0D8903B34E926000EEA22DE
:100E9000EECF06F0EFCF07F006502624026E075083
:100EA0002720036E000E2820046E000E2920056EF8
:100EB00005C084F104C083F103C082F102C081F156
:100EC00048800101928D000184D03F0E3A5C29E1F7
:100ED00001019235000123E28C8E03EE95F0D8904B
:100EE0003B34E926000EEA22EECF06F0EFCF07F002
:100EF00006502624026E07502720036E000E28207D
:100F0000046E000E2920056E05C088F104C087F12B
:100F100003C086F102C085F148800101928F000173
:100F200058D0400E3A5C29E101019331000123E2DF
:100F30008C8C03EE95F0D8903B34E926000EEA2223
:100F4000EECF06F0EFCF07F006502624026E0750D2
:100F50002720036E000E2820046E000E2920056E47
:100F600005C08CF104C08BF103C08AF102C089F185
:100F700048800101938100012CD0410E3A5C29E1A7
:100F8000010193510001E8B223D08C8A03EE95F061
:100F9000D8903B34E926000EEA22EECF06F0EFCFE0
:100FA00007F006502624026E07502720036E000E1D
:100FB0002820046E000E2920056E05C090F104C0A3
:100FC0008FF103C08EF102C08DF14880010193833F
:100FD00000013A682AD0A40E375C0AE13C2803E1FC
:100FE0002EC03CF003D02EC03DF05AD920D01DD0E9
:100FF000B40E375C09E13E2803E12EC03EF003D079
:101000002EC03FF055D911D0C40E375C06E1402800
:1010100003E12EC040F046D908D0D40E375C05E17C
:10102000412803E12EC041F041D948B0FED8120E4C
:10103000345CD8B0E5D03050265C3150275832505F
:10104000285833502958D8A0DAD0338E345209E1C9
:10105000899001014C694B694A6949699191000184
:10106000CDD0010E345C09E18992010150694F69CC
:101070004E694D6991930001C1D0020E345C09E1C3
:10108000899401015469536952695169919500012C
:10109000B5D0030E345C09E189960101586957699E
:1010A0005669556991970001A9D0040E345C09E195
:1010B000899801015C695B695A69596991990001D4
:1010C0009DD0050E345C09E1899A010160695F6970
:1010D0005E695D69919B000191D0060E345C09E167
:1010E0008D9001016469636962696169919D000184
:1010F00085D0070E345C09E18D920101686967694A
:1011000066696569919F000179D0080E345C09E138
:101110008D9401016C696B696A696969929100013A
:101120006DD0090E345C09E18B90010170696F6923
:101130006E696D699293000161D00A0E345C09E119
:101140008B920101746973697269716992950001EA
:1011500055D00B0E345C09E18B94010178697769F5
:10116000766975699297000149D00C0E345C09E1EB
:101170008B9601017C697B697A6979699299000192
:101180003DD00D0E345C09E18C90010180697F69CE
:101190007E697D69929B000131D00E0E345C09E1BD
:1011A0008C9201018469836982698169929D000141
:1011B00025D00F0E345C09E18C9E01018869876996
:1011C00086698569929F000119D0100E345C09E18F
:1011D0008C9C01018C698B698A69896993910001F2
:1011E0000DD0110E345C09E18C9A010190698F6970
:1011F0008E698D699393000101D014D016D812D056
:1012000029AE0FD0296A286A276A266A01EE49F0BA
:10121000480EEE68E82EFDD70101946B936B926B3C
:10122000916B000181787CEF02F03468338E2F6A75
:10123000120E2F5C33E2D8902F34E96EEA6AEA3658
:10124000E936EA36490EE926010EEA22EFCF02F02E
:10125000ECCF03F0ECCF04F0ECCF05F03050025CA3
:1012600031500358325004583350055815E2D89085
:101270002F34E96EEA6AEA36E936EA36490EE9269B
:10128000010EEA22EFCF30F0ECCF31F0ECCF32F0AC
:10129000ECCF33F02FC034F02F2ACAE3489012006D
:1012A0003C68120040681200426812004168120057
:1012B000420E3E5C07E13F5203E1449039D801D031
:1012C000448034D07B0E3E5C30E101EE49F0480EA4
:1012D000EE68E82EFDD7929089909292899292942E
:1012E00089949296899692988998929A899A9690DA
:1012F0008D9096928D9296948D9494908B909492DA
:101300008B9294948B9494968B9695908C909592C6
:101310008C92959E8C9E959C8C9C959A8C9A0101A2
:10132000946B936B926B916B488000013E68120046
:1013300001EE49F0480EEE68E82EFDD792908990B4
:101340009292899292948994929689969298899889
:10135000929A899A96908D9096928D9296948D9469
:1013600094908B9094928B9294948B9494968B9669
:1013700095908C9095928C92959E8C9E959C8C9C31
:10138000959A8C9A0101946B936B926B916B00010F
:101390001200010E0101986F180E976F010ED66FA3
:1013A000E10ED56F020E0201166F860E156F030E49
:1013B000566FD00E556F040E946F210E936FD5C1EA
:1013C00002F0D6C103F097C106F098C107F00650AD
:1013D000025C196E075003581A6E64EC01F01CC0D1
:1013E00011F01BC010F01AC00FF019C00EF011C0A0
:1013F00098F410C097F40FC096F4050E0E5C02E24C
:101400002384000E0401956F020E2F6E0001200E42
:101410002F5CD8B049D02F5062EC01F098C420F076
:1014200097C41FF096C41EF095C41DF0B9EC00F0EF
:101430001CC011F01BC010F01AC00FF019C00EF044
:1014400097C102F098C103F002C019F003C01AF06E
:1014500064EC01F011C020F010C01FF00FC01EF0AE
:101460000EC01DF02BEC00F01CC09CF41BC09BF4C4
:101470001AC09AF419C099F49CC41CF09BC41BF0C8
:101480009AC41AF099C419F007EC01F001EE95F036
:10149000D8902F34E926000EEA2219C0EEFF1AC0B8
:1014A000EFFF2F2AD8A0B2D715C202F016C203F060
:1014B000D5C106F0D6C107F00650025C196E075080
:1014C00003581A6E64EC01F01CC011F01BC010F040
:1014D0001AC00FF019C00EF011C098F410C097F4A4
:1014E0000FC096F4050E0E5C02E22384000E040188
:1014F000956F210E2F6E0001400E2F5CD8B078D072
:1015000098C411F097C410F096C40FF095C40EF073
:101510002F505AEC01F01CC015F01BC014F01AC07B
:1015200013F019C012F0206A1F6A1E6A840E1D6E25
:1015300015C01CF014C01BF013C01AF012C019F033
:1015400029EC00F01CC015F01BC014F01AC013F0F9
:1015500019C012F011C020F010C01FF00FC01EF013
:101560000EC01DF015C01CF014C01BF013C01AF003
:1015700012C019F0B9EC00F01CC011F01BC010F043
:101580001AC00FF019C00EF0D5C102F0D6C103F099
:1015900002C019F003C01AF064EC01F011C020F091
:1015A00010C01FF00FC01EF00EC01DF02BEC00F09D
:1015B0001CC09CF41BC09BF41AC09AF419C099F487
:1015C0009CC41CF09BC41BF09AC41AF099C419F077
:1015D00007EC01F001EE95F0D8902F34E926000ECB
:1015E000EA2219C0EEFF1AC0EFFF2F2AD8A083D736
:1015F00055C202F056C203F015C206F016C207F03B
:101600000650025C196E075003581A6E64EC01F024
:101610001CC011F01BC010F01AC00FF019C00EF062
:1016200011C098F410C097F40FC096F4050E0E5C2C
:1016300002E22384000E0401956F410E2F6E00011B
:10164000600E2F5CD8B078D098C411F097C410F019
:1016500096C40FF095C40EF02F505AEC01F01CC048
:1016600015F01BC014F01AC013F019C012F0206A54
:101670001F6A1E6A850E1D6E15C01CF014C01BF07B
:1016800013C01AF012C019F029EC00F01CC015F0BC
:101690001BC014F01AC013F019C012F011C020F0D2
:1016A00010C01FF00FC01EF00EC01DF015C01CF0C2
:1016B00014C01BF013C01AF012C019F0B9EC00F0FE
:1016C0001CC011F01BC010F01AC00FF019C00EF0B2
:1016D00015C202F016C203F002C019F003C01AF0DE
:1016E00064EC01F011C020F010C01FF00FC01EF01C
:1016F0000EC01DF02BEC00F01CC09CF41BC09BF432
:101700001AC09AF419C099F49CC41CF09BC41BF035
:101710009AC41AF099C419F007EC01F001EE95F0A3
:10172000D8902F34E926000EEA2219C0EEFF1AC025
:10173000EFFF2F2AD8A083D793C202F094C203F000
:1017400055C206F056C207F00650025C196E0750EB
:1017500003581A6E64EC01F01CC011F01BC010F0AD
:101760001AC00FF019C00EF011C098F410C097F411
:101770000FC096F4050E0E5C02E22384000E0401F5
:10178000956F610E2F6E00017F0E2F5CD8B079D05F
:1017900098C411F097C410F096C40FF095C40EF0E1
:1017A0002F505AEC01F01CC015F01BC014F01AC0E9
:1017B00013F019C012F0206A1F6A400E1E6E850ECB
:1017C0001D6E15C01CF014C01BF013C01AF012C01F
:1017D00019F029EC00F01CC015F01BC014F01AC061
:1017E00013F019C012F011C020F010C01FF00FC08C
:1017F0001EF00EC01DF015C01CF014C01BF013C06D
:101800001AF012C019F0B9EC00F01CC011F01BC0A6
:1018100010F01AC00FF019C00EF055C202F056C2F7
:1018200003F002C019F003C01AF064EC01F011C01B
:1018300020F010C01FF00FC01EF00EC01DF02BECEA
:1018400000F01CC09CF41BC09BF41AC09AF419C091
:1018500099F49CC41CF09BC41BF09AC41AF099C460
:1018600019F007EC01F001EE95F0D8902F34E9263D
:10187000000EEA2219C0EEFF1AC0EFFF2F2AD8A0EF
:1018800082D7010E0201986F180E976F010ED66F66
:10189000E10ED56F020E0301166F860E156F030E53
:1018A000566F920E556F040E946F100E936FD5C243
:1018B00002F0D6C203F097C206F098C207F00650B5
:1018C000025C196E075003581A6E64EC01F01CC0DC
:1018D00011F01BC010F01AC00FF019C00EF011C0AB
:1018E00098F410C097F40FC096F4050E0E5C02E257
:1018F0002384000E0401956F020E2F6E0001200E4E
:101900002F5CD8B049D02F5062EC01F098C420F081
:1019100097C41FF096C41EF095C41DF0B9EC00F0FA
:101920001CC011F01BC010F01AC00FF019C00EF04F
:1019300097C202F098C203F002C019F003C01AF077
:1019400064EC01F011C020F010C01FF00FC01EF0B9
:101950000EC01DF02BEC00F01CC09CF41BC09BF4CF
:101960001AC09AF419C099F49CC41CF09BC41BF0D3
:101970009AC41AF099C419F007EC01F002EE95F040
:10198000D8902F34E926000EEA2219C0EEFF1AC0C3
:10199000EFFF2F2AD8A0B2D715C302F016C303F069
:1019A000D5C206F0D6C207F00650025C196E075089
:1019B00003581A6E64EC01F01CC011F01BC010F04B
:1019C0001AC00FF019C00EF011C098F410C097F4AF
:1019D0000FC096F4050E0E5C02E22384000E040193
:1019E000956F210E2F6E0001400E2F5CD8B078D07D
:1019F00098C411F097C410F096C40FF095C40EF07F
:101A00002F505AEC01F01CC015F01BC014F01AC086
:101A100013F019C012F0206A1F6A1E6A840E1D6E30
:101A200015C01CF014C01BF013C01AF012C019F03E
:101A300029EC00F01CC015F01BC014F01AC013F004
:101A400019C012F011C020F010C01FF00FC01EF01E
:101A50000EC01DF015C01CF014C01BF013C01AF00E
:101A600012C019F0B9EC00F01CC011F01BC010F04E
:101A70001AC00FF019C00EF0D5C202F0D6C203F0A2
:101A800002C019F003C01AF064EC01F011C020F09C
:101A900010C01FF00FC01EF00EC01DF02BEC00F0A8
:101AA0001CC09CF41BC09BF41AC09AF419C099F492
:101AB0009CC41CF09BC41BF09AC41AF099C419F082
:101AC00007EC01F002EE95F0D8902F34E926000ED5
:101AD000EA2219C0EEFF1AC0EFFF2F2AD8A083D741
:101AE00055C302F056C303F015C306F016C307F042
:101AF0000650025C196E075003581A6E64EC01F030
:101B00001CC011F01BC010F01AC00FF019C00EF06D
:101B100011C098F410C097F40FC096F4050E0E5C37
:101B200002E22384000E0401956F410E2F6E000126
:101B3000600E2F5CD8B078D098C411F097C410F024
:101B400096C40FF095C40EF02F505AEC01F01CC053
:101B500015F01BC014F01AC013F019C012F0206A5F
:101B60001F6A1E6A850E1D6E15C01CF014C01BF086
:101B700013C01AF012C019F029EC00F01CC015F0C7
:101B80001BC014F01AC013F019C012F011C020F0DD
:101B900010C01FF00FC01EF00EC01DF015C01CF0CD
:101BA00014C01BF013C01AF012C019F0B9EC00F009
:101BB0001CC011F01BC010F01AC00FF019C00EF0BD
:101BC00015C302F016C303F002C019F003C01AF0E7
:101BD00064EC01F011C020F010C01FF00FC01EF027
:101BE0000EC01DF02BEC00F01CC09CF41BC09BF43D
:101BF0001AC09AF419C099F49CC41CF09BC41BF041
:101C00009AC41AF099C419F007EC01F002EE95F0AD
:101C1000D8902F34E926000EEA2219C0EEFF1AC030
:101C2000EFFF2F2AD8A083D793C302F094C303F009
:101C300055C306F056C307F00650025C196E0750F4
:101C400003581A6E64EC01F01CC011F01BC010F0B8
:101C50001AC00FF019C00EF011C098F410C097F41C
:101C60000FC096F4050E0E5C02E22384000E040100
:101C7000956F610E2F6E00017F0E2F5CD8B079D06A
:101C800098C411F097C410F096C40FF095C40EF0EC
:101C90002F505AEC01F01CC015F01BC014F01AC0F4
:101CA00013F019C012F0206A1F6A400E1E6E850ED6
:101CB0001D6E15C01CF014C01BF013C01AF012C02A
:101CC00019F029EC00F01CC015F01BC014F01AC06C
:101CD00013F019C012F011C020F010C01FF00FC097
:101CE0001EF00EC01DF015C01CF014C01BF013C078
:101CF0001AF012C019F0B9EC00F01CC011F01BC0B2
:101D000010F01AC00FF019C00EF055C302F056C300
:101D100003F002C019F003C01AF064EC01F011C026
:101D200020F010C01FF00FC01EF00EC01DF02BECF5
:101D300000F01CC09CF41BC09BF41AC09AF419C09C
:101D400099F49CC41CF09BC41BF09AC41AF099C46B
:101D500019F007EC01F002EE95F0D8902F34E92647
:101D6000000EEA2219C0EEFF1AC0EFFF2F2AD8A0FA
:101D700082D7010E0301986F180E976F010ED66F70
:101D8000E10ED56F020E0401166F860E156F030E5D
:101D9000566F040E556F030E946FD40E936FD5C318
:101DA00002F0D6C303F097C306F098C307F00650BD
:101DB000025C196E075003581A6E64EC01F01CC0E7
:101DC00011F01BC010F01AC00FF019C00EF011C0B6
:101DD00098F410C097F40FC096F4050E0E5C02E262
:101DE0002384000E0401956F020E2F6E0001200E59
:101DF0002F5CD8B049D02F5062EC01F098C420F08D
:101E000097C41FF096C41EF095C41DF0B9EC00F005
:101E10001CC011F01BC010F01AC00FF019C00EF05A
:101E200097C302F098C303F002C019F003C01AF080
:101E300064EC01F011C020F010C01FF00FC01EF0C4
:101E40000EC01DF02BEC00F01CC09CF41BC09BF4DA
:101E50001AC09AF419C099F49CC41CF09BC41BF0DE
:101E60009AC41AF099C419F007EC01F003EE95F04A
:101E7000D8902F34E926000EEA2219C0EEFF1AC0CE
:101E8000EFFF2F2AD8A0B2D715C402F016C403F072
:101E9000D5C306F0D6C307F00650025C196E075092
:101EA00003581A6E64EC01F01CC011F01BC010F056
:101EB0001AC00FF019C00EF011C098F410C097F4BA
:101EC0000FC096F4050E0E5C02E22384000E04019E
:101ED000956F210E2F6E0001400E2F5CD8B078D088
:101EE00098C411F097C410F096C40FF095C40EF08A
:101EF0002F505AEC01F01CC015F01BC014F01AC092
:101F000013F019C012F0206A1F6A1E6A840E1D6E3B
:101F100015C01CF014C01BF013C01AF012C019F049
:101F200029EC00F01CC015F01BC014F01AC013F00F
:101F300019C012F011C020F010C01FF00FC01EF029
:101F40000EC01DF015C01CF014C01BF013C01AF019
:101F500012C019F0B9EC00F01CC011F01BC010F059
:101F60001AC00FF019C00EF0D5C302F0D6C303F0AB
:101F700002C019F003C01AF064EC01F011C020F0A7
:101F800010C01FF00FC01EF00EC01DF02BEC00F0B3
:101F90001CC09CF41BC09BF41AC09AF419C099F49D
:101FA0009CC41CF09BC41BF09AC41AF099C419F08D
:101FB00007EC01F003EE95F0D8902F34E926000EDF
:101FC000EA2219C0EEFF1AC0EFFF2F2AD8A083D74C
:101FD00055C402F056C403F015C406F016C407F049
:101FE0000650025C196E075003581A6E64EC01F03B
:101FF0001CC011F01BC010F01AC00FF019C00EF079
:1020000011C098F410C097F40FC096F4050E0E5C42
:1020100002E22384000E0401956F410E2F6E000131
:10202000600E2F5CD8B078D098C411F097C410F02F
:1020300096C40FF095C40EF02F505AEC01F01CC05E
:1020400015F01BC014F01AC013F019C012F0206A6A
:102050001F6A1E6A850E1D6E15C01CF014C01BF091
:1020600013C01AF012C019F029EC00F01CC015F0D2
:102070001BC014F01AC013F019C012F011C020F0E8
:1020800010C01FF00FC01EF00EC01DF015C01CF0D8
:1020900014C01BF013C01AF012C019F0B9EC00F014
:1020A0001CC011F01BC010F01AC00FF019C00EF0C8
:1020B00015C402F016C403F002C019F003C01AF0F0
:1020C00064EC01F011C020F010C01FF00FC01EF032
:1020D0000EC01DF02BEC00F01CC09CF41BC09BF448
:1020E0001AC09AF419C099F49CC41CF09BC41BF04C
:1020F0009AC41AF099C419F007EC01F003EE95F0B8
:10210000D8902F34E926000EEA2219C0EEFF1AC03B
:10211000EFFF2F2AD8A083D793C402F094C403F012
:1021200055C406F056C407F00650025C196E0750FD
:1021300003581A6E64EC01F01CC011F01BC010F0C3
:102140001AC00FF019C00EF011C098F410C097F427
:102150000FC096F4050E0E5C02E22384000E04010B
:10216000956F610E2F6E00017F0E2F5CD8B079D075
:1021700098C411F097C410F096C40FF095C40EF0F7
:102180002F505AEC01F01CC015F01BC014F01AC0FF
:1021900013F019C012F0206A1F6A400E1E6E850EE1
:1021A0001D6E15C01CF014C01BF013C01AF012C035
:1021B00019F029EC00F01CC015F01BC014F01AC077
:1021C00013F019C012F011C020F010C01FF00FC0A2
:1021D0001EF00EC01DF015C01CF014C01BF013C083
:1021E0001AF012C019F0B9EC00F01CC011F01BC0BD
:1021F00010F01AC00FF019C00EF055C402F056C40A
:1022000003F002C019F003C01AF064EC01F011C031
:1022100020F010C01FF00FC01EF00EC01DF02BEC00
:1022200000F01CC09CF41BC09BF41AC09AF419C0A7
:1022300099F49CC41CF09BC41BF09AC41AF099C476
:1022400019F007EC01F003EE95F0D8902F34E92651
:10225000000EEA2219C0EEFF1AC0EFFF2F2AD8A005
:0622600082D71200FFD737
:020000040030CA
:0300010006160ED2
:020005008580F4
:060008000FC00FE00F40E5
:00000001FF
